:10233B002020202020202020202020200D0A002AD1
:10234B004D3A2053656C6674657374206F6B0D0A80
:10235B00002A573A2053656C667465737420666166
:10236B00696C65640D0A002A52454144590D0A00F7
:10237B0000022F002F2A00AB20015E1601D21102A2
:10238B005A0C02780B02960A02B60902D70802F918
:10239B0007031C06033F05036404038B0303B2020C
:0623AB0003DA0104040046
:10145E00906F157401F0906F15E0FD64126024ED2D
:10146E0075F003A4247BF582E43423F583E493FA28
:10147E00740193FBC3EF9BEE9A4008906F15E00446
:10148E00F080D3ED75F003A4247BF582E43423F5CC
:10149E0083C37401939FFFE4939EFEE4FCFD7BE8FF
:1014AE007A03F9F81204EDC8ECC8C9EDC9CAEECA40
:1014BE00CBEFCB906F15E0FF75F003A4247DF58282
:1014CE00E43423F583E493FDEF75F003A4247AF559
:1014DE0082E43423F583E493C39DFFE49400FEE499
:1014EE00FCFD1204EDECC0E0EDC0E0EEC0E0EFC09C
:1014FE00E0906F15E0FF75F003A42478F582E434D4
:10150E0023F583E493FC740193FDEF75F003A4249B
:10151E007BF582E43423F583C37401939DFFE4933A
:10152E009CFEE4FCFDF8F9CAEECACBEFCBD0E0FF8F
:10153E00D0E0FED0E0FDD0E0FC120578EEC0E0EF8A
:10154E00C0E0906F15E075F003A4247DF582E434BD
:10155E0023F583E493FFE4FCFDFE7BE87A03F9F8C0
:0C156E001204EDD0E02FFFD0E03EFE2282
:1022C200201175906F74E05407906F0CF0C3940363
:1022D2004066E064076061D2117F011230D9E49058
:1022E2006F0CF07F017D127B031231C8301706E5B7
:1022F2006860F980397F017D0E7B031231C8301787
:1023020006E56860F980277F017D0A7B021231C8E9
:10231200301706E56860F98015906F0CE004F0E074
:10232200B403C07F0112319D7F0A1230D9227F028D
:0923320012319D7F0A1230D922FC
:10131E003012030213F8E56864036009E568640B94
:10132E00600302145DD378D5E6954F18E6954E40CE
:10133E000A906F13E4F0A304F0803BAF4FAE4E1251
:10134E00145EEEC0E0EFC0E078D4E6FE08E6FF12D1
:10135E00145ECCEECCCDEFCDD0E0FFD0E0FEC3EDF1
:10136E009FFFEC9EFE906F13F0A3EFF04E70079070
:10137E006F13F0A304F0D201E4906F0CF0906F1392
:10138E00E0FAA3E0FB7C007D0AFFCEEACE12043623
:10139E00906F0CE0240DF582E4346FF583EDF07C54
:1013AE00007D0ACFEBCFCEEACE120436906F13EE4D
:1013BE00F0A3EFF0906F0CE004F0E0B405BF906F77
:1013CE000C7404F0906F0CE0FFF46015740D2FF5A3
:1013DE0082E4346FF583E07008906F0CE014F080B7
:1013EE00E3EF04906F12F0D212227F1E1230D97FDB
:1013FE00017D327B041231C83017043016FA227F79
:10140E000A1230D9906F12E014906F0CF0906F0C9E
:10141E00E0240DF582E4346FF583E0700B7F017DDF
:10142E000B7B041231C88016906F0CE0240DF582F0
:10143E00E4346FF583E0FF7D0B7B011231C830176A
:10144E00043016FA22906F0CE0FF14F0EF70BE22FB
:10214100D2AF122FFD12310B12000E1230301231AC
:10215100FC1231771200031221C81230607BFF7A22
:1021610023793B1200C912316D122C4950107BFFAB
:102171007A23794A1200C97F0112319D800B7BFFBE
:102181007A23795C1200C9D211122024906EE7E003
:10219100FF122BD7122B9E1228EF906EE8E0FEA3C0
:1021A100E0FF122A5E7BFF7A2379721200C9C21204
:1021B100C211301603122F8E12131E906EDFE060D3
:0721C100F11222C280EC22A2
:03000B000223B11C
:1023B100C0E0C0F0C083C082C0D075D008C28CAF6D
:1023C1008CEFFEAD8AED255F78D7F6E55E3E18F617
:1023D100F58C08E6F58AD28CD56309906EDEE0F5BE
:1023E100631227D2D5621B906EDEE0F5620561E5CE
:1023F1006170020560E56145607007E5686003751D
:102401006805E5686404600F1218981226AB121E65
:1024110029122AA1121F87D0D0D082D083D0F0D028
:02242100E032A7
:102A5E00E4FCFDFB7AC079A8F81204ED7BE07A2E37
:102A6E0079007800122A1AC374129FF55FE49EF55E
:102A7E005E906EDEE0F563F562E4F560F561E58982
:102A8E0054F04401F589758CFF758AFFC2B9D2A93D
:032A9E00D28C22B5
:0C312700906EDEE0F562E4F560F56122D8
:1028EF00E5C520E3FB75C50775C50FE5C530E4FBEE
:1028FF00AFC6EF75F004A4FFAEF0E5C5C4131354D3
:10290F00037C002FF53CEC3EF53BE4F53AE53A2528
:10291F00E024C0F8A63B08A63CE53C2527F527E5B3
:10292F003B3526F526053AE53AB40AE1E4F53922B6
:10189800C0D075D008E5C520E3FBE4F5C575C508DB
:1018A800F543754401E5436408700302196DE5C505
:1018B80030E4FB85C62885C53DE5436407600EE531
:1018C800C520E3FBE54304F5C54408F5C5E52875DF
:1018D800F004A4FFAEF0E53DC4131354037C002FBD
:1018E800F546EC3EF545E54325E02429F8A64508EC
:1018F800A646906EDDE055446060AF28122C82AF9A
:101908003D122C82E543B406088545418546428050
:1019180049E54364077043E53925E024C1F8C3E588
:101928002796F527E5261896F526E53925E024C0FB
:10193800F8A64508A646E5462527F527E5453526B0
:10194800F526FEAF277C007D0A1204368E248F25EB
:101958000539E539B40A03E4F5390543E54425E0DA
:10196800F5440218AD300F1EE4A2C492E4A2C59259
:10197800E5A29692E6A29792E72568C4F53EAF3EA7
:0D198800122C82853E40C294D294D0D02211
:10249400C0D075D008300F65906EE7E0FD7C0090E9
:1024A4006EF2E0FB24FFFFE434FFFE120422EF246B
:1024B40001FFE43EFEC3E51F9FF51FE51E9EF51ECA
:1024C4008B3FE53F6021E51EF583E51FF582E0C4FF
:1024D40054F02568C4F0906EE7E0251FF51FE4353D
:1024E4001EF51E153F80DB906EE7E024FFFFE43409
:1024F400FFFEC3E51F9FF51FE51E9EF51ED0D022EB
:0D311A00E4F576F577F578C219122C102235
:1026AB00C0D075D008E56860572019541230C64069
:1026BB004F906EE7E02404906F05F0906F05E0609B
:1026CB003F20133C122D238F7512002E0577E577D3
:1026DB00700205767004E5766480701CF576F577EC
:1026EB000578E578B40C04D21980151230B3E5786F
:1026FB0020E005122C108008906F05E014F080BBD1
:03270B00D0D02209
:102B9E00E4906FB2F0906EF2E075F00584906FB134
:102BAE00F0E4906FB3F0906FAD120650000000008D
:102BBE0074FF78D4F608F6E4906FB4F0F569906F70
:092BCE00ABF0F568A374FFF022DE
:102FE300C0D075D008756801AF68122DB1C29012B8
:0A2FF300311A7F0212319DD0D02266
:0B315700C291906EDEE0906FABF022A2
:0B316200C292906EDEE0906FABF02296
:1011B000C0D075D008E4906F05F020C604E044016B
:1011C000F020C707906F05E04402F0906FACE0FF9D
:1011D000906F05E0FE6F603BEE7025906FBAE0FF08
:1011E00060051231A5802C906FB9E0FF64036004A4
:1011F000EFB404051231A5801A7F0112319D8013CE
:10120000906F05E030E0077F011231A580057F0275
:101210001231A5906F05E0906FACF0300B1EA294D8
:10122000300C01B34016C21A123127906EDBE0FE7B
:10123000A3E0FF122D57122FE302131B201003020D
:10124000131B906EDAE0C4F8540FC868FF906ED993
:10125000E0C454F048FEC3E54D9FFDE54C9EFCE51F
:1012600042C4F8540FC868FFE541C454F048FED3A7
:10127000EF9DEE9C403A906FB2E07006123127026B
:10128000131B906FB1E014F0E0600302131BD21A3D
:10129000906FAD12065000000000E4906FB2F09025
:1012A0006EF2E075F00584906FB1F0123127806B1B
:1012B000906FB1E004F0C21A906FADE0F8A3E0F9CE
:1012C000A3E0FAA3E0FBE8C0E0E542C4F8540FC88D
:1012D00068FFE541C454F048FEC3EF954DFFEE951D
:1012E0004CFE3395E0FDFCD0E0F8EB2FFFEA3EFE2C
:1012F000E93DFDE83CFC906FAD120644906EF2E0D3
:10130000FF906FB2E004F06F7011906EE2E0FEA308
:0E131000E0FF122D57122FE3122494D0D022AA
:101EE200C0D075D008906FADE0F8A3E0F9A3E0FA96
:101EF200A3E0FBE8C0E0E542C4F8540FC868FFE580
:101F020041C454F048FEC3EF954DFFEE954CFE33AD
:101F120095E0FDFCD0E0F8EB2FFFEA3EFEE93DFD47
:101F2200E83CFC906FAD120644300E387F007E0014
:101F32007D007C00906FADE0F8A3E0F9A3E0FAA386
:101F4200E0FBD312060A401C906ED8E0FFD3E56195
:101F52009FE5609400400D123157756802AF681218
:101F62002DB1801E300D1B906EEEE0FEA3E0656188
:101F72007003E5606E700B12315775680AAF681214
:051F82002DB1D0D022BA
:10242300C0D075D008906FABE0600614F07002D294
:1024330091300E3C906EE5E0FEA3E0FFC3E54F9FB5
:10244300FFE54E9EFEC3E5259FE5249E5007E490DD
:102453006FB3F0801B906F03E0FF906FB3E004F065
:102463006F700D123162756803AF68122DB1801E53
:10247300300D1B906EF0E0FEA3E065617003E56034
:102483006E700B12316275680BAF68122DB1D0D02C
:012493002226
:0F30FC00906FABE0600814F07004D291D2922272
:101E2900C0D075D008E5687003021EB7E4F5647583
:101E39006701E56464086065E56425E024F3F582DB
:101E4900E4346EF583E0FEA3E08E65F566F4700375
:101E5900E565F4603EE56955677015E5616566708D
:101E690004E56065657009E5674269AF6412298B0D
:101E7900E5695567601DE5662401FFE43565FEEFF8
:101E890065617003EE6560700AE567F45269AF64D5
:101E99001229D30564E56725E0F5678095C3E52533
:101EA90078D596E52418965005A62408A625E56850
:101EB90014601614601814601A24F9601114601360
:101EC900240B70121211B0800D121EE28008122428
:091ED9002380031230FCD0D0225A
:102BD700CBEFCBEBFD7C007E3A7F98120436CDEB32
:102BE700CD7C001204228E1A8F1B74002FF582EE03
:102BF7003434AF82F5188F197E347F008E1C8F1DF9
:092C07008E1E8F1FD213C214228D
:102C8200201933C213051FE51FAC1E7002051E1466
:102C9200F5828C83EFF0E51F65197004E51E651857
:102CA2007006751E34751F00E51F651D7004E51E54
:072CB200651C7002D2142220
:102D2300C214051DE51DAE1C7002051C14F5828E30
:102D330083E0FFE51D65197004E51C6518700675D1
:102D43001C34751D00E51F651D7004E51E651C70B0
:042D530002D2132273
:102D5700C3E51F9FF51DE51E9EF51CC3E51D9400E9
:102D6700E51C9434400BD3E51D9519E51C951840D7
:0E2D77000CE51B251DF51DE51A351CF51C226B
:101C7C002573202562752025627520257520257514
:101C8C002025752025752025632025627520256368
:101C9C002025632025630D0A00632069676E2025CB
:101CAC007520257520257520257520257520257511
:101CBC002025752025750D0A006320786D69742028
:101CCC00257520256275202562750D0A0063206339
:101CDC0068616E202562750D0A00632067707320A1
:101CEC002562750D0A00696E646578006572617312
:101CFC0065006F6666006F6E002A56455253494F59
:101D0C004E3A20522D4441532056332E370D0A00A3
:101D1C0063210063207264617300632069676E0045
:101D2C006320786D69740063206368616E006320C2
:101D3C0067707300633F006300632000677073205B
:101D4C00007265736574002A453A20756E6B6E6F70
:091D5C00776E20636D640D0A002E
:08000300E4F57EC216C21522CD
:100AF600906F0CEBF0A3EAF0A3E9F0300B13300C87
:100B060008906F297401F0800D906F297402F080AF
:100B160005E4906F29F0906F0CE0FBA3E0FAA3E0E8
:100B2600F91203BA643F6003020BDC906F0FE0F921
:100B3600A3E0FAA3E0906F34C9F0A3EAF0A3E9F0CA
:100B4600906EDEE0906F37F0906EDDE0906F38F0DB
:100B5600906ED9E0FFA3E0906F39CFF0A3EFF0904D
:100B66006EE5E0FFA3E0906F3BCFF0A3EFF0906E51
:100B7600EEE0FFA3E0906F3DCFF0A3EFF0906EF0B4
:100B8600E0FFA3E0906F3FCFF0A3EFF0300F047FBC
:100B96003180027F30906F41EFF0906F29E0906FC7
:100BA60042F03010047F3180027F30906F43EFF0C7
:100BB600300E047F3180027F30906F44EFF0300DAD
:100BC600047F3180027F30906F45EFF07BFF7A1C07
:100BD600797C1200C922906F0CE0FBA3E0FAA3E037
:100BE600F91203BAFF123076500C906F0DE475F0CF
:100BF600011204C180E0E4906F28F0906F0CE0FBD6
:100C0600A3E0FAA3E0F9121688906F28E025E02405
:100C160012F582E4346FF583EEF0A3EFF0906F0CDB
:100C2600E0FBA3E475F0011204D7A9F0FA1203BAA7
:100C3600FF12307650E7906F28E004F0E0B40BBB6B
:100C4600906F13E0906EDEF0906F15E0906EDDF021
:100C5600906F16E0FFA3E0906ED9CFF0A3EFF0906F
:100C66006F18E0FFA3E0906EE5CFF0A3EFF0906F72
:100C76001AE0FFA3E0906EEECFF0A3EFF0906F1CAA
:100C8600E0FFA3E0906EF0CFF0A3EFF0906F1EE0D0
:100C9600FEA3E0FFEE4F24FF920FA3E0FEA3E0FFCA
:100CA600EE4F24FF920BEF64014E7003D38001C315
:100CB600920C906F22E0FEA3E0FFEE4F24FF92100D
:100CC600A3E0FEA3E0FFEE4F24FF920EA3E0FEA3F7
:090CD600E0FFEE4F24FF920D2215
:10179600906F0CEBF0A3EAF0A3E9F01203BA643FF2
:1017A600600302182D7BFF7A1C79A5906EF3E0FF8B
:1017B600A3E0906F34CFF0A3EFF0906EF5E0FFA3B7
:1017C600E0906F36CFF0A3EFF0906EF7E0FFA3E066
:1017D600906F38CFF0A3EFF0906EF9E0FFA3E090A2
:1017E6006F3ACFF0A3EFF0906EFBE0FFA3E0906FAF
:1017F6003CCFF0A3EFF0906EFDE0FFA3E0906F3ECC
:10180600CFF0A3EFF0906EFFE0FFA3E0906F40CF24
:10181600F0A3EFF0906F01E0FFA3E0906F42CFF0EE
:10182600A3EFF01200C922906F0CE0FBA3E0FAA32D
:10183600E0F91203BAFF123076500C906F0DE47582
:10184600F0011204C180E0E4906F0FF0906F0CE09D
:10185600FBA3E0FAA3E0F9121688906F0FE025E0EB
:1018660024F3F582E4346EF583EEF0A3EFF0906F87
:101876000CE0FBA3E475F0011204D7A9F0FA1203F9
:10188600BAFF12307650E7906F0FE004F0E0B4082C
:02189600BB2273
:101D6500906F0CEBF0A3EAF0A3E9F01203BAB43FCD
:101D7500297BFF7A1C79C5906EE0E0FFA3E0906FA8
:101D850034CFF0A3EFF0906EEAE0906F36F0906FED
:101D950004E0906F37F01200C922906F0CE0FBA3AE
:101DA500E0FAA3E0F91203BAFF123076500C906FF7
:101DB5000DE475F0011204C180E0E4906F15F09018
:101DC5006F0CE0FBA3E0FAA3E0F9121688906F15FB
:101DD500E025E0240FF582E4346FF583EEF0A3EF00
:101DE500F0906F0CE0FBA3E475F0011204D7A9F0A5
:101DF500FA1203BAFF12307650E7906F15E004F03F
:101E0500E0B403BB906F0FE0FFA3E0906EE0CFF06E
:101E1500A3EFF0906F12E0906EEAF0906F14E090EF
:041E25006F04F02234
:10270E00906F0CEBF0A3EAF0A3E9F0906F0CE0FBF6
:10271E00A3E0FAA3E0F91203BAB43F127BFF7A1CCE
:10272E0079D9906EEDE0906F34F01200C922906F5F
:10273E000CE0FBA3E0FAA3E0F91203BAFF12307625
:10274E00500C906F0DE475F0011204C180E0906F93
:10275E000CE0FBA3E0FAA3E0F9121688906EEDEF01
:02276E00F02257
:10277000906F0CEBF0A3EAF0A3E9F0906F0CE0FB94
:10278000A3E0FAA3E0F91203BAB43F127BFF7A1C6C
:1027900079E6906EDFE0906F34F01200C922906FFE
:1027A0000CE0FBA3E0FAA3E0F91203BAFF123076C3
:1027B000500C906F0DE475F0011204C180E0906F31
:1027C0000CE0FBA3E0FAA3E0F9121688906EDFEFAD
:0227D000F022F5
:1006F9007B017A6E799A7D20122FAC906F0FEBF007
:10070900A3EAF0A3E9F04A70047F0180027F009018
:100719006F1CEFF0605F7B017A6E7999121688C8B9
:10072900ECC8C9EDC9CAEECACBEFCB906EEBE0FEBF
:10073900A3E0FFE4FCFD1204EDC8ECC8C9EDC9CA89
:10074900EECACBEFCB906EDBE0FEA3E0FFE4FCFD4D
:10075900EB2FFFEA3EFEED39FDEC38FC906F1212EB
:100769000644906EEBE0FEA3E0FFE4FCFD906F16FB
:1007790012064480767B017A6E7999121688C8EC44
:10078900C8C9EDC9CAEECACBEFCB906EE7E0FFE46A
:10079900FCFDFE1204EDC8ECC8C9EDC9CAEECACB0E
:1007A900EFCB906EDBE0FEA3E0FFE4FCFDEB2FFF57
:1007B900EA3EFEED39FDEC38FC906F1212064490CA
:1007C9006F0FE0FBA3E0FAA3E0F9121688C8ECC8A2
:1007D900C9EDC9CAEECACBEFCB906EE7E0FFE4FCE6
:1007E900FDFE1204ED906F16120644906F12E0FCA4
:1007F900A3E0FDA3E0FEA3E0FF780F1206318F7896
:10080900906F12E0FCA3E0FDA3E0FEA3E0FFEE542D
:100819007FFEE48E768F771230B3906F1CE060090B
:10082900E4906F1AF0A3F0800B120026906F1AEE75
:10083900F0A3EFF0E4906F0CF0A3F0906F0CE0FEE2
:10084900A3E0FFE4FCFD906F16E0F8A3E0F9A3E054
:10085900FAA3E0FBC3120620606C123133906F0ECD
:10086900EFF0906F1CE06014906F0EE0FF906F1B2B
:10087900E02FF0906F1AE03400F08018906F1AE0C2
:10088900FEA3E0FF906F0EE0FD122246906F1AEE74
:10089900F0A3EFF0906F0EE0FF1231950577E57741
:1008A900700205767004E57664807009F576F5774F
:1008B90005781230B3906F0DE004F07006906F0C5C
:1008C900E004F0020844906F1CE07013906F1AE086
:1008D900FEA3E0FF1231BB906F1AEEF0A3EFF09088
:1008E9006F1AE0FF123195906F1BE0FF12319522CC
:10308B00D3EF648094B95007EF24D0FEFF8004EF98
:04309B0024A9FF2243
:10199500906F0CEBF0A3EAF0A3E9F0906F1374FFDE
:1019A500F0A3741CF0A374F2F0A3E4F0A37405F0A3
:1019B500122644EF7003122894906F1374FFF0A35E
:1019C500741CF0A374F8F0A3E4F0A37405F0906F11
:1019D5000CE0FBA3E0FAA3E0F9122644EF70041231
:1019E5002D8522906F1374FFF0A3741CF0A374FE71
:1019F500F0A3E4F0A37403F0906F0CE0FBA3E0FA0E
:101A0500A3E0F9122644EF7003C21522906F1374F8
:101A1500FFF0A3741DF0A37402F0A3E4F0A3740215
:101A2500F0906F0CE0FBA3E0FAA3E0F9122644EF77
:101A35007003D21522906F0CE0FBA3E0FAA3E0F946
:101A45001203BAFF122E595043906F0CE0FBA3E02E
:101A5500FAA3E0F99000011203D3FF12308BCDEF0A
:101A6500CD906F0CE0FBA3E0FAA3E0F91203BAFFF7
:101A750012308BEFC454F02DFF906F0FF0122E82B1
:0D1A8500906F0DE475F0021204C180A922DB
:0431EC00122EEC2291
:0A316D007BFF7A1D79051200C922CC
:1008F900906F1374FFF0A3741DF0A3741CF0A3E4AC
:10090900F0A37402F07B017A6E7998122644EF7095
:1009190004120CDF22906F1374FFF0A3741DF0A36F
:10092900741FF0A3E4F0A37406F07B017A6E799842
:10093900122644EF7018906F0F74FFF0A3741DF026
:10094900A3741FF07B017A6E799E120AF622906FCA
:100959001374FFF0A3741DF0A37426F0A3E4F0A3AD
:100969007405F07B017A6E7998122644EF700A7B40
:10097900017A6E799D12179622906F1374FFF0A376
:10098900741DF0A3742CF0A3E4F0A37406F07B01AA
:100999007A6E7998122644EF700A7B017A6E799EF5
:1009A900121D6522906F1374FFF0A3741DF0A374D8
:1009B90033F0A3E4F0A37406F07B017A6E79981200
:1009C9002644EF700A7B017A6E799E12270E2290D7
:1009D9006F1374FFF0A3741DF0A3743AF0A3E4F04D
:1009E900A37405F07B017A6E7998122644EF700A98
:1009F9007B017A6E799D12277022906F1374FFF034
:100A0900A3741DF0A37440F0A3E4F0A37402F07B77
:100A1900017A6E7998122644EF7018906F0F74FF5F
:100A2900F0A3741DF0A37443F07B017A6E799912D7
:100A39000AF622906F1374FFF0A3741DF0A3744596
:100A4900F0A3E4F0A37402F07B017A6E7998122680
:100A590044EF7018906F0F74FFF0A3741DF0A37426
:100A690043F07B017A6E7999120AF622906E98E02A
:100A7900B464041206F922906F1374FFF0A3741D75
:100A8900F0A37448F0A3E4F0A37404F07B017A6E38
:100A99007998122644EF700A7B017A6E799C1219B3
:100AA9009522906F1374FFF0A3741DF0A3744DF099
:100AB900A3E4F0A37405F07B017A6E7998122644B9
:100AC900EF70041231EC22906E98E0B46904121AA6
:100AD9009222906E98E0B4760412316D22906E984D
:0D0AE900E060097BFF7A1D79531200C922DD
:102F8E0010160280107568047F0112319D7F1E128B
:0E2F9E0030D91208F93015E81220B880E3226D
:102CB900C0D0EF20E72CEF640A6027EF640D6011A4
:102CC9007498257EF582E4346EF583EFF0057E80F5
:102CD900117498257EF582E4346EF583E4F0D216FA
:052CE900F57ED0D022B1
:102504002A4D4553534147453A2053746F72696EBF
:102514006720706172616D657465727320696E20E5
:10252400464C4153480D0A002A4D455353414745F3
:102534003A2046696E69736865642073746F7269C2
:102544006E670D0A00000001C001C802000C001BE8
:1025540001000019003C03FFFFFFFFFFFFFFFFFF27
:0D256400FFFFFFFFFFFFFF00000A01000066
:0A317700757C25757D491210292290
:10102900902549E49324FF920BA3E49324FF920CA7
:10103900A3E49324FF9210A3E493906EDDF090252E
:101049004DE49324FF920FE4906EE7F07F80EF6008
:1010590014906EDDE05F6007906EE7E02402F0EF28
:10106900C313FF80E9300F06906EE7E004F0902586
:101079004EE493906EDEF090254FE493906EE4F089
:10108900902550E493FF740193906ED9CFF0A3EFAC
:10109900F0902552E493FF740193906EE5CFF0A38D
:1010A900EFF0906EDEE0FBFD7C007E037FE812042A
:1010B90036906EE8EEF0A3EFF0906EE7E0FA8BF071
:1010C900A4FF906EEBE5F0F0A3EFF0EB1313543FA0
:1010D900906EF2F0FB906F03F0902554E49324FF97
:1010E900920EA3E49324FF920DA3E493FF7401935A
:1010F900906EEECFF0A3EFF0902558E493FF7401C2
:1011090093906EF0CFF0A3EFF090255AE493906E90
:10111900D8F0906EE4E0FF7E00906EEBE0FCA3E077
:10112900FD120422906EDBEEF0A3EFF0EBFF7E00E0
:10113900EAFD7C00120422E02F906EE3F0906EDB52
:10114900E03E906EE2F0E4FFEF25E0245BF582E4F7
:101159003425F583E493FC740193FDEF25E024F332
:10116900F582E4346EF583ECF0A3EDF00FEFB408EB
:10117900D790256BE493FF740193906EE0CFF0A3B1
:10118900EFF090256DE493906EEAF090256EE4936C
:10119900906F04F090256FE493906EEDF0902570B8
:0711A900E493906EDFF022D9
:100CDF00A20BE433857D82857C83F0A20CE433A3E1
:100CEF00F0A210E433857D82857C83A3A3F0906E00
:100CFF00DDE0857D82857C83A3A3A3F0A20FE4337F
:100D0F00FFE57D2404F582E4357CF583EFF0906EEA
:100D1F00DEE0FFE57D2405F582E4357CF583EFF019
:100D2F00906EE4E0FFE57D2406F582E4357CF583E3
:100D3F00EFF0906ED9E0FEA3E0FFE57D2407F5828A
:100D4F00E4357CF583EEF0A3EFF0906EE5E0FEA3C3
:100D5F00E0FFE57D2409F582E4357CF583EEF0A311
:100D6F00EFF0A20EE433FFE57D240BF582E4357C32
:100D7F00F583EFF0A20DE433FFE57D240CF582E45B
:100D8F00357CF583EFF0906EEEE0FEA3E0FFE57D9E
:100D9F00240DF582E4357CF583EEF0A3EFF0906E31
:100DAF00F0E0FEA3E0FFE57D240FF582E4357CF54E
:100DBF0083EEF0A3EFF0906ED8E0FFE57D2411F500
:100DCF0082E4357CF583EFF0E4906F0CF0906F0CBC
:100DDF00E0FF6408603BEF25E024F3F582E4346E16
:100DEF00F583E0FEA3E0FFE57D2412F582E4357C78
:100DFF00F583C083C082906F0CE0D082D08375F0F2
:100E0F0002120681EEF0A3EFF0906F0CE004F08079
:100E1F00BC906EE0E0FEA3E0FFE57D2422F582E4C6
:100E2F00357CF583EEF0A3EFF0906EEAE0FFE57D01
:100E3F002424F582E4357CF583EFF0906F04E0FF16
:100E4F00E57D2425F582E4357CF583EFF0906EED9A
:100E5F00E0FFE57D2426F582E4357CF583EFF09005
:100E6F006EDFE0FFE57D2427F582E4357CF583EF27
:100E7F00F07BFF7A2579041200C9122CEE7BFF7AE2
:070E8F0025792C1200C92295
:10202400E5C520E3FB75C50675C50EE5C530E4FBC3
:10203400AFC6EF75F004A4FFAEF0E5C5C4131354A6
:10204400037C002FF54DEC3EF54CE5C520E3FB7514
:10205400C50775C50FE5C530E4FBAFC6EF75F004E1
:10206400A4FFAEF0E5C5C4131354037C002FF54A56
:10207400EC3EF549F54E854A4FD21AE4F547F5484A
:10208400FFEF25E0247BF582E4346FF583E54CF023
:10209400A3E54DF0E54D2548F548E54C3547F547B2
:1020A4000FEFB410DCE4F54BE5482401F54DE435BD
:0420B40047F54C227E
:1027D200301A5EE5482401F54DE43547F54CE54BEA
:1027E20025E0247BF582E4346FF583E0FEA3E0FF6D
:1027F200C3E5489FF548E5479EF547E54B25E024AC
:102802007BF582E4346FF583E541F0A3E542F0E520
:10281200422548F548E5413547F547054BE54BB4B8
:102822001003E4F54B85494E854A4F852449852599
:022832004A2238
:102FFD00D21B43878075985AE589540F4420F58973
:0A300D00758DFFD28ED2BCD2AC222A
:03002300022E07A3
:102E0700C0E0C0F0C083C082C0D075D01030980732
:102E1700AF99C298122CB9309904C299D21BD0D05D
:092E2700D082D083D0F0D0E0325B
:08319500301BFDC21B8F9922C3
:0731AD00CEEFCE1231952296
:102E3000E5C520E3FB8FC5EF4408F5C5E5C530E4E3
:102E4000FBAFC6EF75F004A4FFAEF0E5C5C41313E5
:092E50005403FDE5F0EF4DFF22F3
:102EEC00E4F5A8F5E8F5B8F5F875780FE578A2E003
:102EFC0092B5A2E192B3A2E292B4A2E392B202FF23
:022F0C00FE22A3
:1030B300E578A2E092B5A2E192B3A2E292B4A2E3D0
:0330C30092B222A4
:0C313300E5764480857782F583E0FF227A
:10002E0090D3557499F090ACAA7466F090D3557431
:10003E0090F0E575F5F0E576D2E7F583E577F58294
:0D004E00E5F0F0E0A2E730F701B340F72243
:102C1000E578A2E092B5A2E192B3A2E292B4A2E377
:102C200092B290D3557499F090ACAA7466F090D398
:102C3000557480F090D3557499F090ACAA7466F0F6
:092C40009080007414F0D21C22F3
:1030C600301C0D908000E020E703D38001C3921CE2
:0330D600A21C2217
:102CEE0075780C122C101230C640FB75780D123010
:102CFE00B3E4F576F577857782857683E0F5751200
:102D0E00002E0577E57770020576E5777004E57697
:052D1E00648070E22258
:0331FC00C21C22D0
:03005B000225710A
:10257100C0E0C0D0C2CC742D25C9F5C9301758159B
:1025810050E5507052E55670128552FCC2C0F551AB
:10259100755601E55425E0F550803CE5566401701F
:1025A1002375FCFFD2C00551E5516553700E3018FB
:1025B10007F556855550801FC217801B7556027549
:1025C10050028013E556B4020E8552FCC2C0755606
:0C25D10001E55425E0F550D0D0D0E032F8
:1030300075FCFFD2C075FE0B75528075EA0DC2FC9F
:08304000D2EC75550AC21722FB
:102EA600C217A202921875FCFFD2C08F53E4F556E2
:102EB600CEEDCE8EFECEEBCE8E54855550EF600213
:032EC600D21722FE
:0631C200D202122EA6222B
:0631C800C202122EA62235
:08319D007D0B7B011231C222FF
:0831A5007D327B041231C222CD
:1030D900C21775FCFFD2C08F55E4F556855550D2FD
:0230E9001722AC
:10157A00413A2534752025347520253475202534C3
:10158A007520253475202534752025347520253499
:10159A007520443A25303262782043433A25632540
:1015AA00632042573A25630D0A002A4D3A20615FAB
:1015BA007374203D2025750D0A002A4D3A206128B2
:1015CA003029203D2025750D0A002A573A20615FEF
:1015DA0073743D25752C2061303D25752028672DB3
:1015EA0073772064697361626C6564290D0A002A45
:1015FA004D3A2070283029203D2025750D0A002AF1
:10160A00573A20502072616E6765205B25752C253C
:10161A00755D0D0A002A573A204257206572726F8B
:10162A0072202842572064697361626C6564290DCF
:10163A000A002A573A206E6F2069676E2025626475
:10164A000D0A002A573A206E6F20786D69740D0AC8
:10165A00002A573A206E6F206770730D0A002A57C6
:10166A003A2064726F677565206572720D0A002AE6
:0E167A00573A206D61696E206572720D0A008C
:0731B400EF60031F80FA2207
:101A92001016028003021B89E4A2C492E0A2C5923E
:101AA200E1A29692E2A29792E3F57BE4FF122E3036
:101AB200EFC0E0EEC0E07F01122E30EFC0E0EEC0DA
:101AC200E07F02122E30EFC0E0EEC0E07F03122E64
:101AD20030EFC0E0EEC0E07F04122E30EFC0E0EE47
:101AE200C0E07F05122E30EFC0E0EEC0E07F0612AC
:101AF2002E30EFC0E0EEC0E07F07122E30906F4232
:101B0200EEF0A3EFF0906F40D0E0F0A3D0E0F090C1
:101B12006F3ED0E0F0A3D0E0F0906F3CD0E0F0A3B5
:101B2200D0E0F0906F3AD0E0F0A3D0E0F0906F38C0
:101B3200D0E0F0A3D0E0F0906F36D0E0F0A3D0E098
:101B4200F0906F34D0E0F0A3D0E0F07BFF7A15790B
:101B52007A906F44E57BF030C6047F6380027F6F2A
:101B6200906F45EFF030C7047F6380027F6F906F04
:101B720046EFF03094047F6F80027F63906F47EFEF
:081B8200F01200C9021A9222C0
:102F6F00A2029293E4F579F57A7F781231B4057A5B
:0F2F7F00E57A70020579E57A640A457970EB22EC
:100E9600E4906F11F0906F0CF0A3F0906F10F0D209
:100EA60002122F6F7F06122E30906F0DE02FF090FA
:100EB6006F0CE03EF0C202122F6F906F10E004F04C
:100EC600E0B420DB906F0CE0FEA3E0FF7C007D2009
:100ED60012048B906F0CEEF0A3EFF07BFF7A15797E
:100EE600B4906F34EEF0A3EFF01200C9E4906F0EE9
:100EF600F0A3F0A3F07F06122E30906F0FE02FF0D4
:100F0600906F0EE03EF0906F10E004F0E0B420E544
:100F1600906F0EE0FEA3E0FF7C007D2012048B9014
:100F26006F0EEEF0A3EFF07BFF7A1579C4906F3465
:100F3600EEF0A3EFF01200C9906F0EE0FEA3E0FF03
:100F4600906F0CE0FCA3E0FDC39FFFEC9EFEC3EF99
:100F5600942DEE64809480502D7BFF7A1579D49081
:100F66006F34ECF0A3EDF0906F0EE0FFA3E0906F0E
:100F760036CFF0A3EFF01200C97F061231A5C210DA
:100F8600906F117406F0E4906F0CF0A3F0906F1060
:100F9600F07F07122E30906F0DE02FF0906F0CE06F
:100FA6003EF0906F10E004F0E0B420E5906F0CE0A6
:100FB600FEA3E0FF7C007D2012048B906F0CEEF008
:100FC600A3EFF07BFF7A1579F9906F34EEF0A3EF7B
:100FD600F01200C9906F0CE0FEA3E0FFC3947DEE13
:100FE60064809482400BD3EF94DBEE64809483405C
:100FF6002C7BFF7A167909906F34EEF0A3EFF0A3FD
:101006007402F0A3747DF0A37403F0A374DBF012F2
:1010160000C97F051231A5906F117405F0906F110C
:03102600E0FF22C6
:101B8A00E4906F0CF0300B1EA294300C01B3401697
:101B9A007BFF7A16791F1200C97F031231A5C20B87
:101BAA00906F0C7403F0E4906F0DF0906F0DE0FFEE
:101BBA006408606AEF25E024F3F582E4346EF58365
:101BCA00E0FCA3E0F47002ECF4604B12313F401FDA
:101BDA007F041231A57BFF7A16793C906F0DE004E1
:101BEA00906F34F01200C9906F0C7404F080279043
:101BFA006F0DE0FF12293F401D7F041231A57BFFC4
:101C0A007A16793C906F0DE004906F34F01200C997
:101C1A00906F0C7404F0906F0DE004F0808D906E5C
:101C2A00E0E07002A3E060201231CE401B7F041274
:101C3A0031A57BFF7A16794D1200C9E4906EE0F067
:101C4A00A3F0906F0C7404F0906EDFE0601E123007
:101C5A001740197F041231A57BFF7A16795B1200AF
:101C6A00C9E4906EDFF0906F0C7404F0906F0CE092
:021C7A00FF2247
:102C4900D201121B8A906FB9EFF06002C201120E15
:102C590096906FBAEFF06002C20120C60B7BFF7A33
:102C69001679681200C9C20120C70B7BFF7A167951
:092C7900791200C9C201A2012276
:10000E00E4FF74B52FF582E4346FF58374FFF00FBF
:05001E00EFB404EE2226
:0C313F00EFC31325E02441FF122FC8222B
:10293F00906F0EEFF0E0FFC31325E02441FF7B0102
:10294F007A6F7910906F177401F0122AE4906F0F5D
:10295F00EFF0906F0EE054012402FF74017E00C867
:10296F00EFC8088005C333CE33CED8F9FF906F1070
:0C297F00E0FDE4EF5D6003D38001C322A3
:10298B00CEEFCEEEC313FF24B5F582E4346FF5839F
:10299B00C083C082E0FDEE5401FC7401C8ECC80892
:1029AB008002C333D8FCF45DD082D083F0EF25E0F6
:1029BB002440FFEEC31324B5F582E4346FAD82FCE3
:0829CB007B01D202122B6322F2
:1029D300CEEFCEEEC313FF24B5F582E4346FF58357
:1029E300C083C082E0FDEE5401FC7401C8ECC8084A
:1029F3008002C333D8FC4DD082D083F0EF25E0248E
:102A030040FFEEC31324B5F582E4346FAD82FC7B43
:072A130001D202122B632225
:10306000E4F57FFF746E2FF582E4346FF583E4F0AE
:063070000FEFB40DEF228A
:10301700906F0E7450F07F587C6F7D0E7B01D2024B
:09302700122B637F50122FC82206
:102E8200906F10EFF0A37450F07F587C6F7D117B30
:102E920001D202122B637F507C6F7D107B01D20224
:042EA200122B63226A
:1020B800906F0E7453F07F587C6F7D0E7B01D202B7
:1020C800122B637F537B017A6F790D906F17740120
:1020D800F0122AE4906F0CEFF0A3E0D394104003C1
:1020E8007410F0906F0DE0604FA37451F07F587C2E
:1020F8006F7D0E7B01D202122B637F517B017A6FB9
:10210800799B906F0DE0906F17F0122AE4906F0C96
:10211800EFF0E4F0906F0DE0FF906F0CE0FE6F6061
:1021280017749B2EF582E4346FF583E0FF12319526
:09213800906F0CE004F080DC2241
:10289400E4906F10F0906F127457F07F587C6F7D46
:1028A400127B01D202122B637F577B017A6F799BD3
:1028B400906F177410F0122AE4906F11EFF0E4F0A7
:1028C400906F11E0FF64106017749B2FF582E4345D
:1028D4006FF583E0FF1231AD906F11E004F080E0FA
:0B28E400906F10E004F0E0B408AB229D
:102D8500906F127456F07F587C6F7D127B01D202D2
:102D9500122B63906F107442F07F567C6F7D107B11
:0C2DA50001D202122B63906F11EFF0229C
:102DB100906F06EFF0906F087454F07F587C6F7D30
:102DC100087B01D202122B637F547C6F7D067B014D
:0B2DD100C202122B63906F07EFF0228C
:102AA100C0D075D008906EDFE06035057F906EDE96
:102AB100E0657F702BF57F906F067455F07F587C31
:102AC1006F7D067B01D202122B637F557B017A6FEA
:102AD1007968906F17740DF0122AE4906F05EFF08A
:032AE100D0D02230
:1021C800D21DE4F557F558F559906EDEE0FF75F02D
:1021D8000A84755C00F55DEFC313755A00F55B90D2
:1021E8006EE0E0FEA3E0FF4E6053906F597404F078
:1021F800E4A3F0FCFDF8F9CAEECACBEFCBFF7EC032
:102208007DA8122A1A7B107A0079007800122A1AFF
:10221800EF14906F5BF0906F04E075F080A4FF906E
:102228006EEAE02F906F5CF0906EEDE0906F5DF0DD
:0E2238007F607C6F7D597B05D202122B6322E2
:0631CE007F60122FC822F1
:1025DD00C0E0A3E558F0A3E559F0A3E52AF0A3E583
:1025ED002CF0A3E52EF0A3E530F0A3E532F0A3E542
:1025FD0034F0A3E536F0A3E538F0A375F000E52936
:10260D0042F0E52B232342F0E52DC442F0E52FC423
:10261D00232345F0F0A375F000E53142F0E53323B7
:10262D002342F0E535C442F0E537C4232345F0F0ED
:07263D00A3E540F0D0E0220C
:101F8700C0D075D008906EE0E07002A3E070030245
:101F97002021301D09E5686005E4F557C21DE557A6
:101FA700FB7A00AC5CAD5DFFCEEACE120436ED4C99
:101FB700705C906EDFE0601DAC5AAD5BCFEBCFCEAF
:101FC700EACE120436ED4C700C906F05741CF0A32A
:101FD7007402F0800A906F05740FF0A37401F090FB
:101FE7006F05E0906F59F0906F06E0906F5AF0120E
:101FF70025DD7F607C6F7D59906F05E0FBC2021283
:102007002B63E56860080559E559700205580557BF
:0D201700906EDEE065577002F557D0D022C4
:102F2F000000CC01D8011400F0013C002800E4019E
:102F3F00A0016C007800B40150009C01880144008E
:050026007EFF7FFF22B8
:10224600CBEFCBCAEECAC9EDC9E9540FFFEAEB6F73
:10225600540F25E0FFE433FE742F2FF582EE342F62
:10226600F583EAC4F854F0C868FEEBC4540F48FF7F
:10227600EE540FFEE4936EFA7401936FFBCFE9CF31
:10228600EFC4540F540FFFEAEF6B540F25E0FFE441
:1022960033FE742F2FF582EE342FF583EAC4F854FB
:1022A600F0C868FEEBC4540F48FFEE540FFEE493EB
:0C22B6006EFA7401936FFBCEEACEFF229B
:0731BB00EEF4FEEFF4FF2229
:10283400FF31F0FF3181FF318BFF2F0EFF31D4FFC9
:102844002EC9FF31DAFF31F4FF3048FF31E0FF2FAA
:102854004FFF309FFF31F8FF31FFFF3200FF32019D
:10286400FF3202FF3203FF3204FF3205FF3206FF5C
:102874003207FF3208FF3209FF320AFF320BFF3101
:10288400E6FF31E6FF31E6FF31E6FF31E6FF31E6F0
:0F310B00D296D29775D8C575DBECD2BDD2AD2266
:102FC800E4F56F8F6DD21ED2DDFF122DDCEF641891
:0B2FD8006004EFB44003D38001C3226B
:102B6300906F13ECF0A3EDF08C838D827880EBFEF5
:102B73006006E0F6A308DEFA8B6F8F6DD21ED2DDFE
:102B830030020DCFEBCF122DDC906F15EFF08005E7
:0B2B9300E4906F15F0906F15E0FF223A
:102AE400906F14EBF0A3EAF0A3E9F0CEEFCEA3E0ED
:102AF400FFF56F8E6DD21ED2DD122DDCE4FE906FD9
:102B040017E06E601D74802EF8E6FD906F14E0FBF4
:102B1400A3E0FAA3E0F98E82758300ED1204000E9F
:032B240080DC2230
:102DDC00CEEFCEE4F56AEE2402FDE433FCE56A6D39
:102DEC007001EC6010756BDDD56BFD201E03AF6EB2
:0B2DFC0022056A80E175D8D57F002217
:0431F00075D8D52297
:0A318100856DDA75D8C5E4F56C22FF
:0A318B00856DDA75D8C5E4F56C22F5
:102F0E00C0D075D010E56F700775D8D5C21E800E73
:102F1E00AF6C056C74802FF8E6F5DA75D8C5D0D095
:012F2E002280
:0631D40075D8D5C21E22D1
:102EC900C0D075D010E56C656F700775D8D5C21E76
:102ED900800EAF6C056C74802FF8E6F5DA75D8C5ED
:032EE900D0D02224
:0631DA0075D8D5C21E22CB
:0431F40075D8E52283
:10304800E56F14600A04700C75D8D5C21E80087527
:08305800D8C1800375D8C52220
:0631E00075D8D5C21E22C5
:102F4F00C0D075D0107480256CF8A6DAE56F140523
:102F5F006C656C700575D8C1800375D8C5D0D0224B
:10309F00C0D075D0107480256CF8A6DA75D8D5C25B
:0430AF001ED0D0223D
:0431F80075D8D5228F
:0131FF0022AD
:0132000022AB
:0132010022AA
:0132020022A9
:0132030022A8
:0132040022A7
:0132050022A6
:0132060022A5
:0132070022A4
:0132080022A3
:0132090022A2
:01320A0022A1
:01320B0022A0
:0631E60075D8D5C21E22BF
:03002B00022B277E
:102B2700C0E0C0F0C083C082C0D075D01085D96E18
:102B3700E5D9131313541F75F003A42434F582E465
:102B47003428F583E493740193FA740293F9120617
:0C2B57008DD0D0D082D083D0F0D0E032FE
:0300000002314B7F
:0C314B00787FE4F6D8FD7581D7022141A1
:1003BA00BB010689828A83E0225002E722BBFE0241
:0903CA00E32289828A83E4932274
:1003D300BB010CE58229F582E5833AF583E02250DF
:1003E30006E92582F8E622BBFE06E92582F8E22229
:0D03F300E58229F582E5833AF583E4932243
:10040000F8BB010DE58229F582E5833AF583E8F032
:10041000225006E92582C8F622BBFE05E92582C8DE
:02042000F222C6
:10042200EFF88DF0A4FFEDC5F0CEA42EFEEC88F01F
:04043200A42EFE22D4
:10043600BC000BBE0029EF8DF084FFADF022E4CCAA
:10044600F875F008EF2FFFEE33FEEC33FCEE9DEC73
:10045600984005FCEE9DFE0FD5F0E9E4CEFD22EDB9
:10046600F8F5F0EE8420D21CFEADF075F008EF2F03
:10047600FFED33FD4007985006D5F0F222C398FDF4
:050486000FD5F0EA2291
:10048B00C2D5EC30E709B2D5E4C39DFDE49CFCEE8C
:10049B0030E715B2D5E4C39FFFE49EFE120436C3CA
:1004AB00E49DFDE49CFC800312043630D507C3E4C5
:0604BB009FFFE49EFE22FB
:1004C100C5F0F8A3E028F0C5F0F8E58215827002C6
:0604D1001583E038F02263
:1004D700A3F8E0C5F025F0F0E582158270021583D8
:0604E700E0C838F0E82235
:1004ED00E88FF0A4CC8BF0A42CFCE98EF0A42CFCAE
:1004FD008AF0EDA42CFCEA8EF0A4CDA8F08BF0A42C
:10050D002DCC3825F0FDE98FF0A42CCD35F0FCEB8A
:10051D008EF0A4FEA9F0EB8FF0A4CFC5F02ECD394F
:0F052D00FEE43CFCEAA42DCE35F0FDE43CFC22BC
:10053C0075F008758200EF2FFFEE33FECD33CDCC76
:10054C0033CCC58233C5829BED9AEC99E5829840F9
:10055C000CF582EE9BFEED9AFDEC99FC0FD5F0D6D6
:10056C00E4CEFBE4CDFAE4CCF9A88222B800C1B900
:10057C000059BA002DEC8BF084CFCECDFCE5F0CB3E
:10058C00F97818EF2FFFEE33FEED33FDEC33FCEB77
:10059C0033FB10D703994004EB99FB0FD8E5E4F932
:1005AC00FA227818EF2FFFEE33FEED33FDEC33FC1F
:1005BC00C933C910D7059BE99A4007EC9BFCE99A13
:1005CC00F90FD8E0E4C9FAE4CCFB2275F010EF2F58
:1005DC00FFEE33FEED33FDCC33CCC833C810D70758
:1005EC009BEC9AE899400AED9BFDEC9AFCE899F893
:0E05FC000FD5F0DAE4CDFBE4CCFAE4C8F92226
:102A1A00C2D5E830E70FB2D5E4C39BFBE49AFAE4E7
:102A2A0099F9E498F8EC30E717B2D5122A50120552
:102A3A0078E4C39BFBE49AFAE499F9E498F88003F2
:102A4A0012057830D50DE4C39FFFE49EFEE49DFD98
:042A5A00E49CFC22DA
:10060A00EB9FF5F0EA9E42F0E99D42F0EC6480C867
:06061A0064809845F02207
:10062000EB9FF5F0EA9E42F0E99D42F0E89C45F030
:0106300022A7
:10063100E8600FECC313FCED13FDEE13FEEF13FFA7
:03064100D8F122CB
:0C064400ECF0A3EDF0A3EEF0A3EFF02229
:10065000A8828583F0D083D08212066712066712C3
:100660000667120667E473E493A3C583C5F0C583E8
:10067000C8C582C8F0A3C583C5F0C583C8C582C8F4
:010680002257
:0C068100A42582F582E5F03583F5832284
:06068D008A838982E473F8
:10005E00E5702434F582E4346FF583E00570229068
:10006E006F31300903906F34E475F0011206B3025C
:10007E0003BA2002E97F2ED2028018EF540F24908B
:10008E00D43440D4FF30060BEF24BFB41A00500313
:10009E002461FFE571600215710574E57470020547
:1000AE007330090E906F31E475F0011206B3EF0252
:1000BE0006930231AD7403D2098003E4C209F570D0
:1000CE00906F311206CAE4F571F573F574E571603F
:1000DE00077F201200A180F5F572C203C202C2048E
:1000EE00C205C207C208C20A12006DFF700D3009A8
:1000FE00057F001200B2AF74AE7322B42561C2D573
:10010E00C20612006DFF24D0B40A00501C75F00A0E
:10011E0020D50DC571A42571F5717002D20580E050
:10012E00C572A42572F57280D724CFB41A00EF5091
:10013E0004C2E5D2060202ACD20380C4D20280BE53
:10014E00D20480BAD2D580B8D20780B27F201200F6
:10015E00A12004077401B5710040F112005EFF1278
:10016E0000A10200DBD20AD208809312005EFB12BD
:10017E00005EFA12005EF94A4B700679787A037BBC
:10018E00FF200433E571602FAF72BF00011F7E00A8
:10019E008E827583001203D360050EEE6F70F1C26E
:1001AE00D5EBC0E0EAC0E0E9C0E0EE1202F0D0E02C
:1001BE00F9D0E0FAD0E0FB1203BAFF60A5EBC0E085
:1001CE00EAC0E0E9C0E01200A1D0E02401F9D0E0DD
:1001DE003400FAD0E0FBE57260DDD572DA80837B05
:1001EE00FF7A0279ECD2048098791080027908C2E5
:1001FE0008C20A8008D2D5790A8004790AC2D5E4E9
:10020E00FAFDFEFF12005EFC7B0820031312005E57
:10021E00FD7B1030020A12005EFE12005EFF7B2094
:10022E00EC3382D592D55013C3E43002069FFFE41F
:10023E009EFEE42003039DFDE49CFCE4CBF8C20388
:10024E00EC700CCFCECDCCE824F8F870F38017C349
:10025E00EF33FFEE33FEED33FDEC33FCEB33FB9966
:10026E004002FB0FD8E9EB300305F8D0E0C448B2EA
:10027E0003C0E00AEC4D4E4F78207B0070C2EAC0FE
:10028E00E01202F2D0F0D0E0200304C4C0E0C4B209
:10029E0003C0F012008AD0F0D5F0EB0200DB12069C
:1002AE00D301795301F758014A4C01464201FB4FE5
:1002BE00020344020349015F4302095501ED460161
:1002CE00ED4501ED47039B50014E2D01522E017558
:1002DE002B01562301732003862A0000016D3F3F38
:1002EE003F00790AA2D5200514300709B91002047F
:1002FE0004B9080104A2D5200802500104200466A6
:02030E00920457
:10031000B571005032C0E07F203005177F30A20455
:1003200072087207500D120347C204C208C2077F49
:1003300030800F300703E9C0E01200A1300703D07E
:10034000E0F9D0E0B571CE3007177F30B9100C124C
:1003500000A17F583006077F788003B90803120098
:10036000A13004057F2D0200A17F20200AF87F2BF9
:100370002008F322920480CF286E756C6C29002D22
:1003800050434958D20312005E3003F8C20378711B
:1003900030D504D2027872F602010C12005E2403FA
:1003A000B405004001E490037F93120092743A1266
:0A03B0000092D2057571040201F7F6
:10307600EFC394094006EFC3940E4004EFB4200357
:05308600D38001C3220C
:102E5900EFC394414006EFC394474018EFC3946110
:102E69004006EFC39467400CEFC394304009EFC3A9
:092E7900943A5003D38001C322F6
:10264400906F10EBF0A3EAF0A3E9F0906F13E0FBB6
:10265400A3E0FAA3E0F91203BAFE906F10E0FBA323
:10266400E0FAA3E0F91203BAFD6E702AED600E9051
:102674006F1674FFF5F01204C145F070037F002259
:10268400906F11E475F0011204C1906F14E475F0B9
:10269400011204C180B5D3EE6480F8ED64809840E3
:0726A400037F01227FFF22EA
:102FAC00E94A4B7001221203BAFF6D700122EF70D7
:0C2FBC0004FBFAF92209E970ED0A80EA32
:10168800906F2AEBF0A3EAF0A3E9F0906F2AE0FB51
:10169800A3E0FAA3E0F91203BAFF123076500C90D7
:1016A8006F2BE475F0011204C180E0D201906F2A1B
:1016B800E0FBA3E0FAA3E0F91203BAFF642B60048D
:1016C800EFB42D1D906F2AE0FBA3E475F00112041E
:1016D800D7A9F0FA1203BA642D6003D38001C3922C
:1016E80001906F2D12065000000000906F2AE0FB59
:1016F800A3E0FAA3E0F91203BAFF1230EB506A7FB5
:101708000A7E007D007C00906F2DE0F8A3E0F9A32D
:10171800E0FAA3E0FB1204EDC8ECC8EDC0E0EEC0AF
:10172800E0EFC0E0906F2AE0FBA3E0FAA3E0F91233
:1017380003BAFF3395E0FEEF24D0FFEE34FFFEE45A
:10174800FCFDD0E0FBD0E0FAD0E0F9EB2FFFEA3E59
:10175800FEED39FDEC38FC906F2D120644906F2B8E
:10176800E475F0011204C18082300110906F2DE001
:10177800FCA3E0FDA3E0FEA3E0FF8011906F2DE045
:0E178800FCA3E0FDA3E0FEA3E0FF1206A522F5
:10069300BB010689828A83F0225002F722BBFE0146
:0206A300F32240
:0E06A500C3E49FFFE49EFEE49DFDE49CFC2266
:1006B300F8E0FBA3A3E0F925F0F0E58215827002D0
:0706C3001583E0FA38F02274
:0906CA00EBF0A3EAF0A3E9F02231
:1006D300D083D082F8E4937012740193700DA3A3B6
:1006E30093F8740193F5828883E4737402936860CA
:0606F300EFA3A3A380DFCA
:1030EB00EFC394304009EFC3943A5003D38001C32C
:0130FB0022B2
:00000001FF
